S01E000062696E2F64656D6F70726F675F73746D3332663736372E737265631F
S315080080000000082049870008998700089987000812
S3150800801099870008998700089987000800000000DA
S31508008020000000000000000000000000998700081A
S31508008030998700080000000099870008D187000882
S315080080409987000899870008998700089987000882
S315080080509987000899870008998700089987000872
S315080080609987000899870008998700089987000862
S315080080709987000899870008998700089987000852
S315080080809987000899870008998700089987000842
S315080080909987000899870008998700089987000832
S315080080A09987000899870008998700089987000822
S315080080B09987000899870008998700089987000812
S315080080C09987000899870008998700089987000802
S315080080D099870008998700089987000899870008F2
S315080080E099870008998700089987000899870008E2
S315080080F099870008998700089987000899870008D2
S3150800810099870008998700089987000899870008C1
S3150800811099870008998700089987000899870008B1
S3150800812099870008998700089987000899870008A1
S315080081309987000899870008998700089987000891
S315080081409987000899870008998700089987000881
S315080081509987000899870008998700089987000871
S315080081609987000899870008998700089987000861
S315080081709987000899870008998700080000000079
S315080081809987000899870008998700089987000841
S315080081909987000899870008998700089987000831
S315080081A09987000899870008998700089987000821
S315080081B09987000899870008998700089987000811
S315080081C09987000899870008000000009987000829
S315080081D099870008998700089987000899870008F1
S315080081E099870008998700089987000899870008E1
S311080081F09987000899870008EE11AA5527
S315080081FC10B5054C237833B9044B13B10448AFF3C7
S3150800820C00800123237010BD7404002000000000B8
S3150800821C1CC10008084B10B51BB108490848AFF338
S3150800822C00800848036803B910BD074B002BFBD028
S3150800823CBDE81040184700BF000000007804002075
S3150800824C1CC10008740400200000000053B94AB988
S3150800825C002908BF00281CBF4FF0FF314FF0FF3034
S3150800826C00F07EB9ADF1080C6DE904CE00F006F805
S3150800827CDDF804E0DDE9022304B070472DE9F04788
S3150800828C8C460E460446089D002B50D18A4217464A
S3150800829C6CD9B2FA82FEBEF1000F0BD0CEF12004D7
S315080082AC20FA04F401FA0EF644EA060C02FA0EF762
S315080082BC00FA0EF44FEA1749220CBCFBF9F01FFA28
S315080082CC87F809FB10C642EA064600FB08F3B342D8
S315080082DC09D9F61900F1FF3280F02281B34240F237
S315080082EC1F8102383E44F61AA2B2B6FBF9F309FB13
S315080082FC136642EA064403FB08F8A04509D9E419B3
S3150800830C03F1FF3280F00A81A04540F20781023B57
S3150800831C3C44C8EB040443EA00400021002D62D01B
S3150800832C24FA0EF400232C606B60BDE8F0878B42B0
S3150800833C07D9002D55D0002185E841000846BDE82F
S3150800834CF087B3FA83F1002940F09080B34202D348
S3150800835C824200F2F880841A66EB03060120B446C2
S3150800836C002D40D085E81010BDE8F08712B901271A
S3150800837CB7FBF2F7B7FA87FEBEF1000F35D1F31B40
S3150800838C4FEA17481FFA87FC0121B3FBF8F0220CB9
S3150800839C08FB103642EA06460CFB00F3B34207D933
S315080083ACF61900F1FF3202D2B34200F2CE80104623
S315080083BCF61AA2B2B6FBF8F308FB136642EA0644B1
S315080083CC0CFB03FCA44507D9E41903F1FF3202D2CE
S315080083DCA44500F2B5801346CCEB040443EA0040EE
S315080083EC9CE729462846BDE8F087CEF1200106FA17
S315080083FC0EF307FA0EF720FA01F94FEA1748CE40A2
S3150800840C49EA0309B6FBF8FA4FEA194408FB1A6657
S3150800841C1FFA87FC44EA06430AFB0CF29A4200FA56
S3150800842C0EF40AD9DB190AF1FF3180F087809A42DB
S3150800843C40F28480AAF1020A3B449B1A1FFA89F976
S3150800844CB3FBF8F108FB113349EA034301FB0CF6BD
S3150800845C9E4207D9DB1901F1FF326BD29E4269D9CC
S3150800846C02393B449B1B41EA0A418EE7C1F1200EB7
S3150800847C22FA0EF48B40234320FA0EF706FA01F47F
S3150800848C4FEA134C26FA0EF63C43B6FBFCF9270CBE
S3150800849C0CFB19661FFA83F847EA064609FB08F728
S315080084ACB74202FA01F200FA01FA08D9F61809F1EC
S315080084BCFF3041D2B7423FD9A9F102091E44F61B37
S315080084CCA0B2B6FBFCF40CFB146640EA064704FBA8
S315080084DC08F8B84507D9FF1804F1FF3028D2B84573
S315080084EC26D9023C1F4444EA0940C8EB0707A0FBFF
S315080084FC02894F4544464E4614D329D065B3BAEB88
S3150800850C040367EB060707FA0EFECB40CF404EEA8C
S3150800851C030385E888000021BDE8F0871346F8E6D2
S3150800852C1046E0E6B8EB020469EB03060138E5E70A
S3150800853C0446D8E7114695E78146C0E78A467CE7A4
S3150800854C023B3C4448E708460AE702383E442FE714
S3150800855CC245E7D33E46D1E72946BDE8F08700BFBA
S3150800856C704700BF70B50F4E0F4D761BB61018BF6F
S3150800857C002405D0013455F8043B9847A642F9D196
S3150800858C0A4E0B4D761B03F0C3FDB61018BF00241C
S3150800859C06D0013455F8043B9847A642F9D170BD6C
S315080085AC70BD00BF68C1000868C1000870C100082A
S315080085BC68C1000870B4840746D0541E002A41D0FE
S315080085CCCDB2034602E0621EE4B3144603F8015B1F
S315080085DC9A07F8D1032C2ED9CDB245EA05250F2CCE
S315080085EC45EA054519D903F110022646103E0F2E09
S315080085FC42F8105C42F80C5C42F8085C42F8045CE1
S3150800860C02F11002F2D8A4F1100222F00F0204F0C3
S3150800861C0F041032032C13440DD91E462246043A75
S3150800862C032A46F8045BFAD8221F22F00302043206
S3150800863C134404F003042CB1C9B21C4403F8011BFF
S3150800864CA342FBD170BC704714460346C2E700BF71
S3150800865C024B13B1024800F005B870470000000041
S3150800866C7D860008002301461A46184600F014B801
S3150800867C38B5074D074C2C1BA41005D0013C55F8F2
S3150800868C043D9847002CF9D1BDE8384003F046BDA7
S3150800869C74C1000870C100082DE9F047254C2568FF
S315080086ACD5F848410646884692469946C4B360684A
S315080086BC1F2817DC431C76B104EB80050122C5F88C
S315080086CC88A0D4F8881182401143022EC4F8881168
S315080086DCC5F808911ED00230636044F8208000204B
S315080086ECBDE8F087144B03B34FF4C870AFF30080A2
S315080086FC0446D0B1D5F84831002780E88800C5F87B
S3150800870C484138460123C4F88871C4F88C71002E88
S3150800871CE1D0D1E7D4F88C110A43C4F88C21DAE7F6
S3150800872C05F5A674C5F84841C1E74FF0FF30BDE81A
S3150800873CF08700BF34C1000800000000DFF834D011
S3150800874C002103E00C4B5B58435004310B480C4B8F
S3150800875C42189A42F6D30B4A02E0002342F8043B2D
S3150800876C094B9A42F9D300F0A7FBFFF7FBFE00F082
S3150800877CD1F970470000082074C100084000002099
S3150800878C7404002074040020D83D0020FEE7000085
S3150800879C08B501F0FBF9084BA3FB0030800901F082
S315080087AC8BFF042001F09EFF002211464FF0FF308C
S315080087BC01F052FF08BD00BFD34D621008B501F099
S315080087CCE5FF08BD08B501F0D5FF01F09DFF08BD12
S315080087DC0C4B1968C1F3072353FA81F3C1F307420B
S315080087EC1A440B0E13FA82F39BB2002205E00549D4
S315080087FC1144087903449BB20132372AF7D95842F7
S3150800880C80B270470000002008B5FFF7E1FF044B63
S3150800881C9B8F984201D0002008BD012008BD00BFDF
S3150800882C0000002008B5064B1A68064B9A4203D17D
S3150800883CFFF7EAFF10B908BD002008BD012008BDE6
S3150800884C00000020A2E742CE08B5FFF7C1FF014B96
S3150800885C988708BD0000002008B5FFF7E3FF68B944
S3150800886C074A084B1A60002304E0064A1A440021FA
S3150800887C11710133372BF8D9FFF7E6FF08BD00BF96
S3150800888CA2E742CE0000002038B504460D46FFF795
S3150800889CC9FF40B1372C08D8054B1C442571FFF786
S315080088ACD3FF012038BD002038BD002038BD00BFDD
S315080088BC0000002010B500F039FAFFF77FFF00F52D
S315080088CCFA70134B1860FFF779FF42F210730344E2
S315080088DC104A136002F094F80F4A00231380538051
S315080088EC0E4A138053800E4A138053804EF60300AB
S315080088FC02F0C6F800F056FA0A4C204600F066FA62
S3150800890C0621204603F07CFA03F098FA10BD00BF46
S3150800891C9C04002090040020503700204C3700207F
S3150800892C483700209404002008B50B4B1B7813F02D
S3150800893C400F0FD113F0020F0CD0084B1B681A7995
S3150800894CFF2A07D15B792BB901210020FFF79CFF81
S3150800895C01F090FF08BD00BF143700201C3700201B
S3150800896C10B500F043FA48B3384A1080384B9C8946
S3150800897C4FF4006002F09EF884420DD1012002F0FB
S3150800898CD3F8324B1B88CBB103F052F800F058FAE7
S3150800899C00222E4B1A8011E02D4B9C8940F60600BE
S315080089AC02F088F8844209D102F0D2FF274B1B88C3
S315080089BC23B100F045FA0022244B1A80FFF7FEFE7D
S315080089CC244B1B68984233D303F5FA73214A136078
S315080089DC002414E0C4EB04135A001F4B13441F4A1B
S315080089EC1360022002F0A0F8184B1B8833B103F071
S315080089FC1FF800F025FA0022144B1A800134002CBB
S31508008A0CE8D0002412E0164B03EB8413154A1360C6
S31508008A1C052002F089F80D4B1B8833B103F008F8D2
S31508008A2C00F00EFA0022094B1A800134002CEAD009
S31508008A3CFFF7C4FE0C4B1B68984206D342F2107221
S31508008A4C1A44094B1A6002F051FF10BD0837002072
S31508008A5C543700209C04002024370020203700209F
S31508008A6C983D0020183700209004002000B595B0DA
S31508008A7C214B1A6C42F080521A641B6C03F080531B
S31508008A8C0093009B1D4B1A6842F440421A601B68FF
S31508008A9C03F440430193019B012307934FF480335E
S31508008AAC089302230D934FF480020E9208220F921C
S31508008ABC4FF4D87210921193129307A800F04AFD3E
S31508008ACC00B1FEE701F088F800B1FEE70F23029328
S31508008ADC02230393002304934FF4A05305934FF4F6
S31508008AEC80530693072102A800F09AFF00B1FEE70F
S31508008AFC15B05DF804FB00BF00380240007000405A
S31508008B0C08B501F02BFEFFF7B1FFFFF741FE01F0A8
S31508008B1C57FE08BD08B5FFF7F3FFFFF79DFEFFF7F5
S31508008B2CC9FE01F0A3FE00210846FFF7ADFE01F0D1
S31508008B3C51FEFFF715FF01F0FBFEF8E710B58EB0F6
S31508008B4C484B1A6C42F080521A641A6C02F0805226
S31508008B5C0192019A5A6C42F480425A645A6C02F495
S31508008B6C80420292029A1A6B42F001021A631A6B3D
S31508008B7C02F001020392039A1A6B42F002021A637C
S31508008B8C1A6B02F002020492049A1A6B42F004025F
S31508008B9C1A631A6B02F004020592059A1A6B42F0D4
S31508008BAC08021A631A6B02F008020692069A1A6BE6
S31508008BBC42F040021A631A6B02F040020792079AB7
S31508008BCC1A6C42F480221A641B6C03F480230893F3
S31508008BDC089B032001F02EFD002211466FF00B00B6
S31508008BEC01F03AFD002211466FF00A0001F034FD3F
S31508008BFC002211466FF0090001F02EFD00221146E5
S31508008C0C6FF0040001F028FD002211466FF00300F6
S31508008C1C01F022FD002211466FF0010001F01CFD47
S31508008C2C002211464FF0FF3001F016FD8023099300
S31508008C3C01230A9300240B940C9409A90A4801F001
S31508008C4C0BF84FF44073099302230A930B940323EE
S31508008C5C0C9307230D9309A9044800F0FDFF0EB0E9
S31508008C6C10BD00BF0038024000040240000C024050
S31508008C7C0268294B9A424ED1F0B589B0A3F59043B8
S31508008C8C1A6B42F000721A631A6B02F000720092A9
S31508008C9C009A1A6B42F080621A631A6B02F08062B1
S31508008CAC0192019A1A6B42F000621A631B6B03F06D
S31508008CBC00630293029B3223039302270497002630
S31508008CCC0596032506950B24079403A9134800F06B
S31508008CDCC3FF86230393049705960695079403A961
S31508008CEC0F4800F0B9FF4FF4005303930497059609
S31508008CFC0695079403A90B4800F0AEFF4FF42053D2
S31508008D0C0393049705960695079403A9064800F05D
S31508008D1CA3FF09B0F0BD704700800240000802406E
S31508008D2C00000240000402400018024010B5164B21
S31508008D3C08221A7000225A70272199706921D97055
S31508008D4C5B21197145215971104C1149216001217A
S31508008D5C616022826361A261E2614FF400032362BF
S31508008D6C204601F01DFB04230A4A0B49204601F054
S31508008D7C59F90423094A0A49204601F08DF9204677
S31508008D8C01F036FC10BD00BFA0040020EC1E00202C
S31508008D9C00800240341F00201C0600209C06002080
S31508008DAC6C1E0020074A1178074B197051785970B8
S31508008DBC91789970D178D9701179197152795A714B
S31508008DCC704700BFA004002078050020064B1A78CF
S31508008DDC02705A7842709A788270DA78C2701A7968
S31508008DEC02715B7943717047A004002038B51248AC
S31508008DFC01F01AFAE8B9104DAC8F2246296C0F48C7
S31508008E0C03F07BF92A6B136843F0004313600023C5
S31508008E1CAB632B6841F214029A5812F0800F09D0F2
S31508008E2C802141F214029950002141F2080299500E
S31508008E3C00E00024204638BDEC1E002054370020E4
S31508008E4C38B5184BDC6AFFF7B9FC00F1FA0503E0F4
S31508008E5CFFF7B4FC854204D32368002BF8DB012307
S31508008E6C00E0002363B1104B1D880E4CE36A2A46BA
S31508008E7C0E49986803F041F92946204601F042F953
S31508008E8C084B1B6841F214029A5812F0200F07D0AF
S31508008E9C202141F214029950002141F20402995002
S31508008EAC38BD00BFEC1E00200837002054370020C0
S31508008EBC08B5FFF783FC08BD0C4AD2F8883043F492
S31508008ECC7003C2F888300A4B1A6842F001021A601D
S31508008EDC002199601868074A02401A60064A5A60C7
S31508008EEC1A6822F480221A60D960704700ED00E0F7
S31508008EFC00380240FFFFF6FE10300024704700BF12
S31508008F0C2DE9F04105460F4616469846069C1EE086
S31508008F1CB4F1FF3F1BD02CB101F038FCC8EB0000B4
S31508008F2C844214D82A68136823F4D07313602A6809
S31508008F3C936823F001039360202385F8693085F83C
S31508008F4C6A30002385F868300320BDE8F0812B6869
S31508008F5CDB6937EA03030CBF01230023B342D7D0DE
S31508008F6C0020BDE8F08100BF2DE9F04182B01E4615
S31508008F7C90F86A30DBB2202B71D104460D46904628
S31508008F8C002A18BF00296CD090F86830012B6AD0DB
S31508008F9C012380F868300023C366222380F86A30E0
S31508008FAC01F0F4FB0746A4F85880A4F85A80A36885
S31508008FBCB3F5805F0AD1236923B940F2FF13A4F8ED
S31508008FCC5C301AE0FF23A4F85C3016E04BB9236931
S31508008FDC1BB9FF23A4F85C300FE07F23A4F85C30A0
S31508008FEC0BE0B3F1805F08D123691BB97F23A4F882
S31508008FFC5C3002E03F23A4F85C30B4F85C8022E0D5
S3150800900CB4F85A309BB2013B9BB2A4F85A3000967E
S3150800901C3B46002220212046FFF772FF28BBA36897
S3150800902CB3F5805F08D1236933B923685B6A08EA0C
S3150800903C030325F8023B06E023685B6A5FFA88F2AD
S3150800904C13402B700135B4F85A309BB2002BD7D18C
S3150800905C202384F86A30002084F8680006E0022091
S3150800906C04E0012002E0022000E0032002B0BDE883
S3150800907CF08100BF38B50446826803691A43436910
S3150800908C1A43C3691A4301680868A34B0340134380
S3150800909C0B6021684B6823F44052E36813434B601A
S315080090ACA269236A1A4321688B6823F43063134335
S315080090BC8B602568994B9D4213D103F59433D3F8ED
S315080090CC903003F00303032B03D8DFE803F0D40630
S315080090DC04081023E0E00223DEE00423DCE0082386
S315080090ECDAE08F4B9D4218D103F5FA33D3F890305A
S315080090FC03F00C030C2B08D8DFE803F0BF070707AF
S3150800910C0B070707090707070D001023C4E00223FE
S3150800911CC2E00423C0E00823BEE0824B9D4218D16E
S3150800912C03F5F833D3F8903003F03003102B0CD03A
S3150800913C03D8002B00F0A38003E0202B03D0302BA0
S3150800914C05D01023A8E00223A6E00423A4E00823F4
S3150800915CA2E0754B9D4218D103F5F633D3F890303F
S3150800916C03F0C003402B0CD003D8002B00F08980E9
S3150800917C03E0802B03D0C02B05D010238CE00223F0
S3150800918C8AE0042388E0082386E0684B9D421AD1BE
S3150800919C03F5F433D3F8903003F44073B3F5807FBA
S315080091AC0DD002D8002B6ED005E0B3F5007F04D0A5
S315080091BCB3F5407F05D010236EE002236CE0042340
S315080091CC6AE0082368E05A4B9D421AD103F592339C
S315080091DCD3F8903003F44063B3F5806F0DD002D802
S315080091EC002B52D005E0B3F5006F04D0B3F5406FF1
S315080091FC05D0102350E002234EE004234CE008234C
S3150800920C4AE04C4B9D4219D103F5E033D3F8903024
S3150800921C03F44053B3F5805F0CD001D8BBB305E01B
S3150800922CB3F5005F04D0B3F5405F05D0102333E0E7
S3150800923C022331E004232FE008232DE03E4B9D4208
S3150800924C27D103F5DE33D3F8903003F44043B3F556
S3150800925C804F0CD001D8F3B105E0B3F5004F04D01C
S3150800926CB3F5404F05D0102316E0022314E004236F
S3150800927C12E0082310E001230EE000230CE0002383
S3150800928C0AE0002308E0002306E0012304E000239B
S3150800929C02E0102300E00023E269B2F5004F59D131
S315080092AC082B4DD8DFE803F005101B4C244C4C4C0E
S315080092BC2F0000F071FC63685A0802EB4000B0FB03
S315080092CCF3F39BB200203DE000F076FC63685A0885
S315080092DC02EB4000B0FBF3F39BB2002032E062686D
S315080092EC164B03EB5203B3FBF2F39BB2002029E0B7
S315080092FC00F030FB63685A0802EB4000B0FBF3F34E
S3150800930C9BB200201EE06268530803F58033B3FB5A
S3150800931CF2F39BB2002015E0F369FFEF0010014051
S3150800932C0044004000480040004C004000500040FB
S3150800933C0014014000780040007C00400048E80119
S3150800934C0120002323F00F02C3F3420313432268C0
S3150800935CD36038BD082B3BD8DFE803F005101B3A61
S3150800936C253A3A3A300000F017FC636800EB5300D4
S3150800937CB0FBF3F080B2E860002038BD00F01CFCAE
S3150800938C636800EB5300B0FBF3F080B2E860002092
S3150800939C38BD62680F4B03EB5203B3FBF2F39BB277
S315080093ACEB60002038BD00F0D5FA636800EB53007B
S315080093BCB0FBF3F080B2E860002038BD6268530851
S315080093CC03F50043B3FBF2F39BB2EB60002038BD08
S315080093DC012038BD0024F400436A13F0010F06D0AF
S315080093EC01684B6823F40032836A13434B60436A63
S315080093FC13F0020F06D001684B6823F48032C36A57
S3150800940C13434B60436A13F0040F06D001684B688C
S3150800941C23F48022036B13434B60436A13F0080F43
S3150800942C06D001684B6823F40042436B13434B6028
S3150800943C436A13F0100F06D001688B6823F4805228
S3150800944C836B13438B60436A13F0200F06D00168B5
S3150800945C8B6823F40052C36B13438B60436A13F077
S3150800946C400F11D001684B6823F48012036C134328
S3150800947C4B60036CB3F5801F06D101684B6823F467
S3150800948CC002436C13434B60436A13F0800F06D03B
S3150800949C01684B6823F40022836C13434B607047B6
S315080094AC10B582B004460023C36601F06FF9226832
S315080094BC126812F0080F0AD06FF07E430093034629
S315080094CC00224FF400112046FFF71AFD40B920235D
S315080094DC84F8693084F86A30002084F8680000E063
S315080094EC032002B010BD00BF80B310B5044690F837
S315080094FC693013F0FF0F04D1002380F86830FFF7AA
S3150800950CFDFC242384F869302268136823F00103D0
S3150800951C13602046FFF7AEFD012819D0636A13B114
S3150800952C2046FFF759FF2268536823F4904353608B
S3150800953C2268936823F02A0393602268136843F021
S3150800954C010313602046FFF7ABFF10BD01207047DF
S3150800955C10BD00BF002800F0D78170B582B0044654
S3150800956C036813F0010F65D0A64B9B6803F00C0338
S3150800957C042B0AD0A34B9B6803F00C03082B0DD1C4
S3150800958CA04B5B6813F4800F08D09E4B1B6813F432
S3150800959C003F4FD06368002B4CD1B7E16368B3F535
S315080095AC803F05D1974A136843F48033136020E053
S315080095BC4BB9944B1A6822F480321A601A6822F452
S315080095CC80221A6015E0B3F5A02F09D18D4B1A68C5
S315080095DC42F480221A601A6842F480321A6008E053
S315080095EC884B1A6822F480321A601A6822F4802290
S315080095FC1A6063687BB101F0C9F8054605E001F00D
S3150800960CC5F8401B642800F283817E4B1B6813F453
S3150800961C003FF4D00EE001F0B9F8054605E001F07C
S3150800962CB5F8401B642800F27581764B1B6813F459
S3150800963C003FF4D1236813F0020F54D0714B9B688A
S3150800964C13F00C0F0AD06F4B9B6803F00C03082B16
S3150800965C16D16C4B5B6813F4800F11D1694B1B68E0
S3150800966C13F0020F03D0E368012B40F05581654ACD
S3150800967C136823F0F803216943EAC103136032E047
S3150800968CE368E3B15F4A136843F00103136001F022
S3150800969C7DF8054605E001F079F8401B022800F232
S315080096AC3D81584B1B6813F0020FF4D0554A1368CA
S315080096BC23F0F803216943EAC103136013E0514A06
S315080096CC136823F00103136001F060F8054605E002
S315080096DC01F05CF8401B022800F22281494B1B68FA
S315080096EC13F0020FF4D1236813F0080F2AD063691C
S315080096FCA3B1444A536F43F00103536701F046F88C
S3150800970C054605E001F042F8401B022800F20A81E2
S3150800971C3C4B5B6F13F0020FF4D013E0394A536FCE
S3150800972C23F00103536701F031F8054605E001F013
S3150800973C2DF8401B022800F2F780324B5B6F13F0B2
S3150800974C020FF4D1236813F0040F00F083802D4B1D
S3150800975C1B6C13F0805F0BD12A4B1A6C42F08052AB
S3150800976C1A641B6C03F080530193019B012500E0DE
S3150800977C0025254B1B6813F4807F13D1224A1368E6
S3150800978C43F48073136001F001F8064605E000F017
S3150800979CFDFF801B642800F2C9801B4B1B6813F461
S315080097AC807FF4D0A368012B05D1164A136F43F0BA
S315080097BC010313671FE04BB9124B1A6F22F0010213
S315080097CC1A671A6F22F004021A6714E0052B09D1DE
S315080097DC0C4B1A6F42F004021A671A6F42F0010218
S315080097EC1A6708E0074B1A6F22F001021A671A6FFC
S315080097FC22F004021A67A368B3B100F0C7FF064645
S3150800980C0CE000BF003802400070004000F0BEFFBC
S3150800981C801B41F28833984200F28A804C4B1B6FAE
S3150800982C13F0020FF2D00FE000F0B0FF064606E088
S3150800983C00F0ACFF801B41F2883398427AD8444B2F
S3150800984C1B6F13F0020FF3D125B1414A136C23F0A9
S3150800985C80531364A369002B6ED03D4A926802F0BC
S3150800986C0C02082A6AD0022B39D1394A136823F01C
S3150800987C8073136000F08AFF054604E000F086FF4B
S3150800988C401B02285CD8324B1B6813F0007FF5D1BD
S3150800989CE269236A1343626A43EA8213A26A52088C
S315080098AC013A43EA0243E26A43EA0263226B43EA59
S315080098BC0273274A5360136843F08073136000F0F1
S315080098CC65FF044604E000F061FF001B022839D846
S315080098DC1F4B1B6813F0007FF5D0002035E01C4A9F
S315080098EC136823F08073136000F050FF044604E0FD
S315080098FC00F04CFF001B022826D8154B1B6813F0EA
S3150800990C007FF5D1002020E00120704701201CE0E3
S3150800991C03201AE0032018E0012016E0032014E0C7
S3150800992C032012E0032010E003200EE003200CE0D5
S3150800993C03200AE0032008E0002006E0012004E0EA
S3150800994C032002E0032000E0032002B070BD00BF34
S3150800995C0038024038B52F4B9B6803F00C03042BD8
S3150800996C55D0082B01D02C4838BD2A4B5A6802F022
S3150800997C3F025B6813F4800F20D0264B5B68C3F359
S3150800998C8813DC000025690141EAD4616001041BD7
S3150800999C61EB0505A90141EA9461A001001B61EB85
S315080099AC0501C01841F100014B0243EAD0534402A9
S315080099BC204619460023FEF749FC1FE0154B5B6849
S315080099CCC3F38813DC000025690141EAD461600100
S315080099DC041B61EB0505A90141EA9461A001001B72
S315080099EC61EB0501C01841F100018B0243EA905363
S315080099FC8402204619460023FEF728FC054B5B68B3
S31508009A0CC3F3014301335B00B0FBF3F038BD0348E5
S31508009A1C38BD00BF003802400024F40000127A005A
S31508009A2C002800F09C8070B50446544B1B6803F064
S31508009A3C0F038B420BD2514A136823F00F030B43C7
S31508009A4C1360136803F00F03994240F08A80236869
S31508009A5C13F0020F17D013F0040F04D0484A93687A
S31508009A6C43F4E0539360236813F0080F04D0444A78
S31508009A7C936843F4604393604148836823F0F0028B
S31508009A8CA368134383600D46236813F0010F2ED089
S31508009A9C6268012A05D13A4B1B6813F4003F0DD1B5
S31508009AAC61E0022A05D1364B1B6813F0007F05D1FD
S31508009ABC5BE0334B1B6813F0020F58D030498B68A8
S31508009ACC23F0030313438B6000F060FE064606E0A2
S31508009ADC00F05CFE801B41F28833984249D8284B2B
S31508009AEC9B6803F00C036268B3EB820FF0D1234B2F
S31508009AFC1B6803F00F039D420AD2204A136823F011
S31508009B0C0F032B431360136803F00F039D4232D1E6
S31508009B1C236813F0040F06D019498B6823F4E05216
S31508009B2CE36813438B60236813F0080F07D0144AB5
S31508009B3C936823F46043216943EAC1039360FFF7F2
S31508009B4C09FF0F4B9B68C3F303130E4AD35CD8402B
S31508009B5C0D4B1860002000F0DBFD002070BD0120C5
S31508009B6C7047012070BD012070BD012070BD012019
S31508009B7C70BD032070BD012070BD00BF003C0240C3
S31508009B8C0038024038C1000868040020014B1868E8
S31508009B9C704700BF6804002008B5FFF7F7FF044BB1
S31508009BAC9B68C3F38223034AD35CD84008BD00BF25
S31508009BBC0038024048C1000808B5FFF7E7FF044B18
S31508009BCC9B68C3F34233034AD35CD84008BD00BF35
S31508009BDC0038024048C1000810B582B01C4B1A6CFC
S31508009BEC42F080521A641B6C03F080530193019B5C
S31508009BFC184A136843F48033136000F0C7FD044613
S31508009C0C05E000F0C3FD001BB0F57A7F1AD8114B9E
S31508009C1C5B6813F4803FF4D00E4A136843F40033A0
S31508009C2C136000F0B3FD044605E000F0AFFD001B21
S31508009C3CB0F57A7F08D8074B5B6813F4003FF4D06D
S31508009C4C002002E0032000E0032002B010BD00BF94
S31508009C5C0038024000700040F0B583B00024D8E00C
S31508009C6C0123A3400A6803EA0205AB4240F0D08000
S31508009C7C4A68122A18BF022A10D1E608083650F884
S31508009C8C26C004F0070297000F22BA402CEA020EEF
S31508009C9C0A69BA404EEA020240F8262002686700B2
S31508009CAC0326BE40F64302EA060E4A6802F0030291
S31508009CBCBA404EEA020202604A6802F1FF3E112AD5
S31508009CCC18BFBEF1010F01D9122A10D1826806EA13
S31508009CDC020ECA68BA404EEA02028260426822EA5A
S31508009CEC03034A68C2F30012A2401A434260C368CF
S31508009CFC1E408B68BB403343C3604B6813F0805FD0
S31508009D0C00F08680454B5A6C42F480425A645B6C70
S31508009D1C03F480430193019BA608B21C404B53F8ED
S31508009D2C227004F003039B000F229A4027EA0207CD
S31508009D3C3C4A904225D002F58062904223D002F527
S31508009D4C8062904221D002F5806290421FD002F5C3
S31508009D5C806290421DD002F5806290421BD002F5BB
S31508009D6C8062904219D002F58062904217D002F5B3
S31508009D7C8062904215D002F58062904213D1092276
S31508009D8C12E0002210E001220EE002220CE003226F
S31508009D9C0AE0042208E0052206E0062204E007226F
S31508009DAC02E0082200E00A2202FA03F33B430236D9
S31508009DBC1B4A42F826301C4B1A68EB4302EA030688
S31508009DCC4F6817F4803F01D045EA0206164A16601A
S31508009DDC526803EA02064F6817F4003F01D045EAB9
S31508009DEC0206114A5660926803EA02064F6817F48F
S31508009DFC801F01D045EA02060B4A9660D2681340CA
S31508009E0C4E6816F4001F01D045EA0203064AD360D1
S31508009E1C01340F2C7FF624AF03B0F0BD0038024096
S31508009E2C0038014000000240003C01400AB1816143
S31508009E3C70470904816170475079137943EA002306
S31508009E4C07480B50D07893781B0443EA0063507884
S31508009E5C43EA002312781343024A8B50704700BF1B
S31508009E6C4080024044800240016841F218028B5837
S31508009E7C43F400538B507047016841F218028B5813
S31508009E8C43F002038B50704770B59EB0044629B157
S31508009E9C4FF40063C3604FF480438360E3691BB9D6
S31508009EAC4FF48063079301E0002307932068036847
S31508009EBC354A1A40A168E3681943079B0B4343F4D8
S31508009ECC00731343036023681D68012000F064FCCB
S31508009EDC23681D60236840225A6023685D68012048
S31508009EEC00F05AFC23685D60236800259D60236892
S31508009EFCDD602268936923F0BE031B041B0C43F038
S31508009F0C8003936123689E69012000F045FC236851
S31508009F1C9E612368DD612368DD69012000F03CFC45
S31508009F2C2368DD61216841F218054B59174A1A4016
S31508009F3C174B13434B5123685E59012000F02CFC38
S31508009F4C23685E51236803F58053124A1A60236806
S31508009F5C03F580531D68012000F01EFC236803F5E9
S31508009F6C80531D60A369012B06D1216841F21C029E
S31508009F7C8858094B03438B50626900212046FFF72A
S31508009F8C5BFF1EB070BD00BF0F8120FF233FDEF8BC
S31508009F9C040020028020C1024000010010B582B0E6
S31508009FAC0446002301930268136843F00803136000
S31508009FBC03681B680193012000F0EEFB2368019AE5
S31508009FCC1A6002B010BD00BF10B582B0044600235B
S31508009FDC01930268136843F00403136003681B6853
S31508009FEC0193012000F0D8FB2368019A1A6002B08D
S31508009FFC10BD00BF30B583B0054600230193026837
S3150800A00C41F21804135943F48013135103681B596E
S3150800A01C0193012000F0C0FB2B68019A1A5103B07A
S3150800A02C30BD00BFF0B490F84540012C30D0012467
S3150800A03C80F84540022480F84440C162002419E0A7
S3150800A04C65014F194FF480164E5140F2F45606FB33
S3150800A05C0426BE60C6691EB94E5946F440064E51D2
S3150800A06C5D1EAC4204D2651C01EB4515FD6000E093
S3150800A07CF96001349C42E3D3026841F21003D150D3
S3150800A08C012380F84430002380F84530184600E058
S3150800A09C0220F0BC704700BFF0B490F84540012C84
S3150800A0AC2DD0012480F84540022480F84440816272
S3150800A0BC002416E066018D194FF000478F5144F2C3
S3150800A0CCF4566E6040F2F45606FB0426AE605E1E2D
S3150800A0DCB44204D2661C01EB4616EE6000E0E96059
S3150800A0EC01349C42E6D3026841F20C03D150012399
S3150800A0FC80F84430002380F84530184600E00220EA
S3150800A10CF0BC704790F84530012B00F08480012391
S3150800A11C80F84530022380F8443039B9012380F899
S3150800A12C4430002280F8452018467047C36A1A68DE
S3150800A13C002A07DA122380F84430002380F84530C9
S3150800A14C0120704730B440F2F45291420AD9344C8B
S3150800A15CA4FB0124A40A40F2F45202FB141212B115
S3150800A16C013400E00124012C3AD11A6842F040521D
S3150800A17C1A60C36AC1F30C015960C26A136843F0CA
S3150800A18C00431360C36ADB68C3622CE0C56A2A689D
S3150800A19C22F040522A6023B9C56A2A6842F08052D6
S3150800A1AC2A60C26A40F2F4555560621E93420DD17C
S3150800A1BCC56A2A6842F000522A601A4A02FB04123F
S3150800A1CC02F2F452C56AC2F30C026A60C56A2A68BE
S3150800A1DC42F000422A60C26AD268C262013300E0C9
S3150800A1EC00239C42D2D8036841F214029A5812F002
S3150800A1FC040F08D0042141F2140299500268002178
S3150800A20C41F20403D150012380F84430002380F82E
S3150800A21C4530184601E00220704730BC704700BF35
S3150800A22C0BB002AC0CFAFFFF90F84530012B3FD06F
S3150800A23C012380F84530022380F84430836A1A6873
S3150800A24C002A2DDB1A6812F4807F18D0826B013233
S3150800A25C8263012A00D1036343631A68C2F30D4271
S3150800A26C043AC263026B92680264DB688362012358
S3150800A27C80F84430002380F84530184670471A6831
S3150800A28C12F4007F07D00363002242630122826323
S3150800A29CDB68836204E0826B01328263DB6883626B
S3150800A2AC012380F84430002280F845201846704770
S3150800A2BC02207047F8B590F84430DBB2822B33D0C5
S3150800A2CC16460546822380F844300268146904F061
S3150800A2DC1C04038ADB029BB21C43890101F4F86156
S3150800A2EC0C4344F00104146100F050FA07460FE0E1
S3150800A2FC00F04CFAC01BB0F5803F07D3012385F854
S3150800A30C4430002385F845300320F8BD2B681C69BA
S3150800A31C14F0010FECD12B685B699BB233600123F7
S3150800A32C85F844300020F8BD0220F8BD90F844307A
S3150800A33CDBB2422B32D070B50546422380F8443046
S3150800A34C0068046904F01C042B8ADB029BB21C43CC
S3150800A35C890101F4F8610C4344F0030492B242619A
S3150800A36C2B681C6100F012FA06460FE000F00EFA94
S3150800A37C801BB0F5803F07D3012385F844300023B2
S3150800A38C85F84530032070BD2B681C6914F0010F45
S3150800A39CECD1012385F84430002070BD02207047AB
S3150800A3AC70B582B000230193002800F0088104469A
S3150800A3BC90F8443013F0FF0F04D1002380F8453091
S3150800A3CCFEF756FC804B5A6C42F480425A645B6C1E
S3150800A3DC03F480430093009B7C4B5A6822F40002DA
S3150800A3EC5A605968226A0A435A60236803F58053EF
S3150800A3FC1A6842F001021A6000F0C8F905460CE02A
S3150800A40C00F0C4F9401BB0F5FA7F06D9032584F889
S3150800A41C4450002384F84530D2E0236803F5805273
S3150800A42C126812F0010FEBD11D6925F01C05FFF718
S3150800A43CADFB674B0344674A934202D845F00805BF
S3150800A44C16E0654B0344654A934202D845F00C0561
S3150800A45C0EE0634B0344634A934209D9624B0344A7
S3150800A46C624A934202D845F0040501E045F010050E
S3150800A47C23681D614FF4004200212046FFF756FF62
S3150800A48C054638B101212046FFF7FEFC012584F864
S3150800A49C445095E0FF2000F07FF96368002B6ED0DE
S3150800A4AC00F074F9064601AA01212046FFF702FFBF
S3150800A4BC00F06CF9801B41F2883398420BD90121C4
S3150800A4CC2046FFF7E1FC012384F84430002384F886
S3150800A4DC4530032574E0019B13F0040FE3D04FF4C9
S3150800A4EC805200212046FFF721FF38B10121204672
S3150800A4FCFFF7CAFC012584F8445061E000F046F9E0
S3150800A50C064601AA01212046FFF7D4FE00F03EF9C3
S3150800A51C801B41F2883398420BD901212046FFF75C
S3150800A52CB3FC012384F84430002384F84530032512
S3150800A53C46E0019B13F0200FE3D001AA1021204618
S3150800A54CFFF7B8FE38B101212046FFF79DFC01251F
S3150800A55C84F8445034E0019B13F0040F03D04FF4F5
S3150800A56C0062E26001E00022E26013F0020F02D002
S3150800A57C0023A3601BE04FF48043A36017E0E36855
S3150800A58CC3F3CF02A368C3F34F031A430021204633
S3150800A59CFFF7CCFE38B101212046FFF775FC0125E3
S3150800A5AC84F844500CE040F6FF7000F0F5F80021F2
S3150800A5BC2046FFF769FC012384F8443000E00125A6
S3150800A5CC284602B070BD00BF003802400038014072
S3150800A5DC00D3CEFEBFE1E40040F1E9FD3F787D01F2
S3150800A5EC00796CFCFF596202001F0AFA7FF0FA0226
S3150800A5FC38B590F84530012B1AD00446012580F859
S3150800A60C4550022380F84430FFF7C8FC2046FFF774
S3150800A61CDBFC2046FFF7EEFC2046FFF725FC204620
S3150800A62CFFF72AFC84F84450002084F8450038BD0E
S3150800A63C022038BD064AD36823F4E0631B041B0CBE
S3150800A64C000200F4E0601843024B0343D3607047E2
S3150800A65C00ED00E00000FA0530B4144BDB68C3F3D8
S3150800A66C0223C3F10704042C28BF04241D1D062D40
S3150800A67C01D9DD1E00E00025012303FA04F4013C90
S3150800A68C2140A940AB40013B1A400A43002806DA90
S3150800A69C00F00F001201D2B2054B1A5403E0120156
S3150800A6ACD2B2044B1A5430BC704700BF00ED00E020
S3150800A6BC14ED00E000E400E00138B0F1807F0AD226
S3150800A6CC064B5860F021064A82F823100020986041
S3150800A6DC07221A6070470120704700BF10E000E09F
S3150800A6EC00ED00E0042805D1054A136843F004037D
S3150800A6FC13607047024A136823F00403136070470B
S3150800A70C10E000E0704700BF08B5FFF7FBFF08BD77
S3150800A71C10B504460E4B18784FF47A73B3FBF0F366
S3150800A72C0C4A1068B0FBF3F0FFF7C6FF58B90F2CAC
S3150800A73C0BD8002221464FF0FF30FFF78DFF064B52
S3150800A74C1C60002010BD012010BD012010BD00BFEB
S3150800A75C70040020680400206C04002008B503204F
S3150800A76CFFF768FF0020FFF7D3FFFEF7E7F9002095
S3150800A77C08BD00BF034A1368034909780B441360E4
S3150800A78C704700BF0437002070040020014B18687E
S3150800A79C704700BF0437002038B50446FFF7F6FFAC
S3150800A7AC0546B4F1FF3F02D0044B1B781C44FFF757
S3150800A7BCEDFF401B8442FAD838BD00BF7004002058
S3150800A7CC08B5002280210248FFF730FB08BD00BF00
S3150800A7DC0004024010B5FDF7F1FF0E4B1B68C31AB7
S3150800A7ECB3F5FA7F14D304460B4B1B783BB90122FD
S3150800A7FC094B1A7080210948FFF718FB06E000225E
S3150800A80C054B1A7080210548FFF710FB014B1C609D
S3150800A81C10BD00BFA8040020AC04002000040240B0
S3150800A82C08B50948094B03604FF46143436000239C
S3150800A83C8360C36003610C2242618361C361036256
S3150800A84C4362FEF751FE08BDB404002000480040E0
S3150800A85C08B50023012201460348FEF785FB08B913
S3150800A86C012008BD002008BDB404002008B5FFF778
S3150800A87CD7FF08BDBFF34F8F0549CA6802F4E062DB
S3150800A88C044B1343CB60BFF34F8F00BFFDE700BFEC
S3150800A89C00ED00E00400FA0508B5214B1B78ABB9AE
S3150800A8AC2048FFF7D5FF012838D11E4B1B78013BF2
S3150800A8BCDBB23F2B32D8FDF781FF1B4B1860012208
S3150800A8CC174B1A700022194B1A7008BD174B1B78B8
S3150800A8DC013314481844FFF7BBFF012814D1134A57
S3150800A8EC13780133DBB213700E4A1278934215D1E2
S3150800A8FC00220B4B1A700B4B5B78FF2B0ED1094BB6
S3150800A90C9B785BB9FFF7B6FFFDF758FF064B1B683C
S3150800A91C6433984202D90022014B1A7008BD00BF55
S3150800A92C6905002028050020B00400202405002015
S3150800A93C08B5FFF7B1FF08BD10B4013A0A440BE09D
S3150800A94C0C784B7803EB04239BB2184480B28342F1
S3150800A95C01D9013080B202319142F1D307D10B787B
S3150800A96C1B02184480B2834201D9013080B25DF8CB
S3150800A97C044B704770B4C5780D44EDB2134CE570B2
S3150800A98C83780E0A3344DBB2A3704278627000787F
S3150800A99C20709CB2A64206D90132D2B20B4C627018
S3150800A9AC0AB901302070C9B28D420CDA0133DBB218
S3150800A9BC064A93703BB953780133DBB2537013B91B
S3150800A9CC13780133137070BC704700BF1037002022
S3150800A9DC10B5094C2368014603F10800FFF7CAFFB6
S3150800A9EC2368064A117819725178597291789972B6
S3150800A9FCD278DA7210BD00BF20370020103700203D
S3150800AA0C00221A4B1A7006E00021194A22F8131074
S3150800AA1C0133164A1370154B1B78002BF4D0002201
S3150800AA2C124B1A7009E0C3EB03114A0011490A4488
S3150800AA3C0021517601330D4A13700C4B1B78002BF1
S3150800AA4CF1D04FF480620C4B1A800022074B1A7017
S3150800AA5C07E00A4A02EB8312002191800133034A6C
S3150800AA6C1370024B1B78002BF3D070477605002029
S3150800AA7C443700202437002074050020983D002018
S3150800AA8C00220A4B1A700BE01946094A32F81320B1
S3150800AA9C1AB9074B23F8110070470133034A137090
S3150800AAAC024B1B78002BEFD0704700BF76050020B1
S3150800AABC44370020030A43EA002080B2704700BFDF
S3150800AACC08B5142205490020FFF736FF10B1FFF729
S3150800AADCF1FF08BD4FF6FF7008BD00BF62370020B6
S3150800AAEC38B50D4D2C7C6B7C03EB0424143CA4B2BA
S3150800AAFC2044082205F11A0180B2FFF71DFF2246F1
S3150800AB0C05F12201FFF718FF10B1FFF7D3FF38BD87
S3150800AB1C4FF6FF7038BD00BF5437002008B5062025
S3150800AB2CFFF7DEFF08BD00BF70B5A54B1C680428EF
S3150800AB3C00F07181A34BA44A1360A44A136003283E
S3150800AB4C10D1637E03F00F03032B40F0D285238AC2
S3150800AB5C002B40F0CE8508229D4B1A70FDF7E4FEBB
S3150800AB6C00F08CBC02287BD19A4AD3780133DBB22D
S3150800AB7CD37063B993780133DBB293703BB95378CE
S3150800AB8C0133DBB2537013B91378013313700023F6
S3150800AB9C914A1380914A1380637E052B18BF072BA5
S3150800ABAC0AD1A37E0133DBB2A376782B40F0A185BC
S3150800ABBC0023637600F09DBD002B00F09A85228A4F
S3150800ABCC002A41D0A27E511EA176002A40F091851A
S3150800ABDCE27E082A05D0591EC9B201290ED8052AC3
S3150800ABEC0CD1002363768022794B1A70FDF79CFEF4
S3150800ABFC14227B4B83F82F2000F00CBD042A03D8B3
S3150800AC0C03219140C9B200E03021A1760132E276E7
S3150800AC1C03F00F03013B072B00F26B85DFE813F0FB
S3150800AC2C740208000D00EA036905EA036905EA03DC
S3150800AC3C00226B4B83F82F206AE20422644B1A70AD
S3150800AC4CFDF772FE00F04FBC03F00F03032B40F028
S3150800AC5C508508225E4B1A70FDF766FE00F00EBC96
S3150800AC6C052817D15F4B1B689B88002B00F0418584
S3150800AC7C0023534A13605C4A53490A6053490A60D5
S3150800AC8C564A1380544A13800822514B1A7001F005
S3150800AC9C21FAC0E0524B9B7B452B40F02A85504A43
S3150800ACAC157C537C03EB05214B4A1288914200F321
S3150800ACBC20858DB2484B1D80494B1B7D13F03F0FE9
S3150800ACCC40F01785464B5B7D002B40F01285474BB1
S3150800ACDC1C880CB95B885BB1414BDB8B9C4240F002
S3150800ACEC08853F4B1A8C414B5B889A4240F001858C
S3150800ACFCFFF7E6FE4FF6FF73984240F0FA84384B9E
S3150800AD0CDB7D062B00F0B880112B23D0012B40F0ED
S3150800AD1CF084334B93F82230082B40F0EA84304BFE
S3150800AD2C002283F822209B8C4FF6F672934203D9A5
S3150800AD3C09332B4A938402E00833294A9384284B17
S3150800AD4C5A8BDA839A8B1A845C83284A52889A839C
S3150800AD5C00F0CBBC1C3D204B1D80254A214B1A60AC
S3150800AD6C26E09A880AB31E49898C8A421DD1DA884C
S3150800AD7C32B11B49498C8A4202D0B2F58A4F14D19A
S3150800AD8C1A8812B95988002936D04FF6FF718A42AB
S3150800AD9C02D1588888422FD01149498B8A4204D14E
S3150800ADAC0F4A918B5A88914226D040330D4A13602C
S3150800ADBC0C4B1B680F4A9342D3D300F09ABC00BFC6
S3150800ADCC203700208A3700201C3700200C3700203B
S3150800ADDC143700207005002008370020963D002007
S3150800ADEC54370020183700207E37002050370020B3
S3150800ADFC983D0020D83D00200023AC4A1360022160
S3150800AE0CAB4A1170AB4AAC490A60AC490A60AC4A09
S3150800AE1C138001F05FF9AA4B1A88002A00F069849E
S3150800AE2C02F11C0189B2A74B1980A74B080A1874A2
S3150800AE3C5974A6490968087A98751120D875083284
S3150800AE4C92B2100A40EA0222DA84002283F82820F9
S3150800AE5C83F829208A885A84CA889A849C4A108836
S3150800AE6C588352889A830A88DA834A881A8436332E
S3150800AE7C914A136000F024BCFFF750FE4FF6FF739F
S3150800AE8C984240F03684934C17E0617EA1B18E4B04
S3150800AE9C9A8CA3889A420FD18B4B5A8CE3889A4288
S3150800AEAC0AD1894B5A8B23889A4205D1864B9A8BA1
S3150800AEBC63889A4200F046811E34864B9C42E4D93C
S3150800AECC814B93F82F3003F03F03022B14D17E4BA2
S3150800AEDC9B8C99B2804A13800022804B1A7007E02B
S3150800AEEC7F4A32F8132091425BD001337B4A1370A8
S3150800AEFC7A4B1B78002BF3D0734B93F82F3013F047
S3150800AF0C040F40F0F683704B142283F82F20282167
S3150800AF1C6C4A1180502283F82E2093F8290093F856
S3150800AF2C2D2083F8292093F8281093F82C2083F8E1
S3150800AF3C282083F82C1093F8272093F82B4083F8B5
S3150800AF4C274083F82B2093F82640644D2C7093F8F1
S3150800AF5C2A5083F8265083F82A400130C0B283F869
S3150800AF6C2D0068B94B1CDBB2574981F82C303BB91C
S3150800AF7C531CDBB281F82B3013B9013481F82A4003
S3150800AF8C514B5A8C54490A80998C59849A845A8BF9
S3150800AF9CDA839A8B1A844E4A1188598352889A8373
S3150800AFAC79E300244D4B1C701CE019461E224948B7
S3150800AFBC02FB0302527E1AB91E2404FB010415E097
S3150800AFCC072A0CD13CB11E22424902FB0312917E80
S3150800AFDCA27E914203D93F4A1E2404FB0324013363
S3150800AFEC3E4A13703D4B1B78002BDED0002C00F02C
S3150800AFFC80832E4B1C600323A37623760023A3752C
S3150800B00C0422E275E376304DAB8CA3806B8CE3801F
S3150800B01C6B8B2380AB8B638001206076314B1A785F
S3150800B02C22735A7862739A78A273DB78E373208258
S3150800B03C95F82930E37295F82830A37295F82730DD
S3150800B04C637295F826302372FFF7C2FC95F82E002A
S3150800B05C00F0F003502B57DD0022204B1A704BE002
S3150800B06C03F13602184DAA5C002A4DD0012A03D1E9
S3150800B07C01331A4A13703FE0022A35D103F137021D
S3150800B08C114DAA5C042A2FD101F13803EA5C393137
S3150800B09C6B5C43EA0222104B1A8040F20A63934215
S3150800B0AC28BF13466382A3822EE000BF20370020F8
S3150800B0BC143700207E3700201C3700200C37002060
S3150800B0CC963D0020083700205437002018370020FA
S3150800B0DC50370020243700206A050020760500200A
S3150800B0EC443700207005002003F13702A6498A5C14
S3150800B0FC52B11344A54A1370A44B1B78194602097E
S3150800B10C053AB3EB820FABDB10229F4B83F82F204B
S3150800B11C9D4B93F82F2042F0020283F82F2002222F
S3150800B12C83F83620042283F83720062283F8382041
S3150800B13C0A2283F839202C21954A1180602283F83B
S3150800B14C2E206EE2934B1C600022934B1A708E4B8A
S3150800B15C93F82F2012F0040F07D0002363762022D1
S3150800B16C8D4B1A70FDF7E0FBC3E2874B93F82E3034
S3150800B17C1B099B0085480370EB1A143B9BB2844849
S3150800B18C038001F00F01022903D102F03F011229B5
S3150800B19C0FD013B912F0030F0BD07B4BD98C238924
S3150800B1AC994240F03382784B198D6389994240F065
S3150800B1BC2D8212F0100F47D0218A002944D004F1B1
S3150800B1CC0C00FFF7D7FB704B93F82A30734A1078AC
S3150800B1DC834239D16C4B93F82B3051788B4233D14F
S3150800B1EC694B93F82C30927893422DD1664B93F891
S3150800B1FC2D506A4BDB789D4226D120736173A2735E
S3150800B20CE373E37ECBB9237EA27E9B1ADBB2A17DC8
S3150800B21CA3EBD103DBB25AB21944C9B2A175002A01
S3150800B22C01DA5B425AB2E37DA2EB930253FA82F23D
S3150800B23CD3B2E37503EBD10323760122564B1A706E
S3150800B24C237EA37600232382617E01F00F03013B44
S3150800B25C072B00F24E82DFE813F008002300A70044
S3150800B26C7301A301BF01D90165014B4B1B7813F080
S3150800B27C010F00F03E82032363764022464B1A7078
S3150800B28C00232382424B188820B14222424B1A7063
S3150800B29CFFF79EFB0022424B1A80FDF745FBEDE0BB
S3150800B2AC3D4B1B7813F0010F63D0374B93F82F30B7
S3150800B2BC03F03F03122B5CD1334B93F82E0000F0AE
S3150800B2CCF003502B37DD0022304B1A702BE003F1BC
S3150800B2DC36022D4DAA5C72B3012A03D101332B4ACF
S3150800B2EC137020E0022A16D103F13702264DAA5C08
S3150800B2FC042A10D101F13803EA5C39316B5C43EA54
S3150800B30C0222284B1A8040F20A63934228BF13463E
S3150800B31C6382A3820FE003F137021B498A5C52B1A0
S3150800B32C13441A4A1370194B1B7819460209053A25
S3150800B33CB3EB820FCBDB03236376134B93F82620F0
S3150800B34C227293F82720627293F82820A27293F837
S3150800B35C2930E3720120FFF73BFB42220E4B1A7091
S3150800B36C002323820A4A13800D4A1380FDF7DCFA60
S3150800B37C84E02022084B1A70FDF7D6FA054B1B6899
S3150800B38C00225A76B8E500BF54370020760500200F
S3150800B39C08370020203700201437002010370020EB
S3150800B3AC963D00206A050020914B93F82F3013F038
S3150800B3BC010F24D011F0100F21D1238A002B40F055
S3150800B3CC98818C4D2888013080B2FFF701FB8A4A98
S3150800B3DC137843F0100313702A881AB143F002034A
S3150800B3EC854A1370FDF7A0FA012323820823637696
S3150800B3FC0023E37611227E4B83F82F200AE113F003
S3150800B40C200F10D07A4890F834301A0290F835305C
S3150800B41C43EA0200794D2E68304428607548134378
S3150800B42C0288D31A0380734B188848B111F0100F91
S3150800B43C06D1714A137843F002031370FFF7C8FA62
S3150800B44C6B4A92F8301092F8313003EB01239BB219
S3150800B45C6B4A1380A28A934200D80BB9684B1A80A0
S3150800B46C674B1B886382644B1B7813F0030F00F041
S3150800B47C40810022634B1A80FDF756FA5E4B1B7807
S3150800B48C13F0200F08D000235E4A1380637614222B
S3150800B49C574B83F82F20BDE013F0100F0CD0002368
S3150800B4AC584A13800122228204226276E3761122FC
S3150800B4BC4F4B83F82F20ADE0524A12888AB113F00D
S3150800B4CC010F01D000232382238A43B9638A9A4247
S3150800B4DC01D94C4A13804B4B1B88238201E0494AFD
S3150800B4EC13800023E376484B1A68444B1A60454B85
S3150800B4FC1B884BB1238A3BB128333E4A138018224A
S3150800B50C3B4B83F82F2088E03B4B1B7813F0020F3C
S3150800B51C00F0EF802822374B1A801022344B83F820
S3150800B52C2F207AE0344B1B7813F0010F00F0E180E2
S3150800B53C002363761022304B1A70FDF7F5F9D8E024
S3150800B54C2C4B188808B1FFF743FA294B93F82F3080
S3150800B55C13F0010F15D0284B1B7813F0010F05D0EB
S3150800B56C072363760023A376238201E006236376FA
S3150800B57C0120FFF72DFA10221F4B1A70FDF7D4F98C
S3150800B58C44E01D4B1B7813F0010F04D0052363769A
S3150800B59C00232382ADE0174B1B88002B36D1A8E07D
S3150800B5AC144B188808B1FFF713FA114B93F82F3080
S3150800B5BC13F0010F0CD0072363760023A376012022
S3150800B5CCFFF706FA10220C4B1A70FDF7ADF91DE0C1
S3150800B5DC084B1B88D3B98CE0074B1B7813F0010F6B
S3150800B5EC00F08780072363760023A37681E000BFEB
S3150800B5FC5437002008370020143700201C37002049
S3150800B60C6A050020963D00200C37002010223C4B82
S3150800B61C83F82F2028223B4B1A805022384B83F86C
S3150800B62C2E20227A364B83F82A20627A83F82B202E
S3150800B63CA27A83F82C20E27A83F82D20227B83F8D1
S3150800B64C2620627B83F82720A27B83F82820E27BBE
S3150800B65C83F829200622DA75A2885A84E2889A8405
S3150800B66C294A1188598352889A832288DA836288F0
S3150800B67C1A84637E13F0100F06D0214B002283F830
S3150800B68C312083F8302006E01D4B062283F8302043
S3150800B69C0A2283F831201A4C4023A375194B1B88B0
S3150800B6AC1A0A22746374002384F8353084F834300B
S3150800B6BC84F8323084F83330FFF730FAC0436086AA
S3150800B6CC0F4C4523A3730022E273627522750F494A
S3150800B6DC0B8801339BB20B80190AA174E37422768A
S3150800B6EC6276FFF7EDF9C04320830022084B1A70E7
S3150800B6FC70BD0023034A1380054A137070BD00BF42
S3150800B70C5437002008370020503700206C050020DD
S3150800B71C14370020F8B505460E46254A138801331A
S3150800B72C9BB21380B3F5FA4F03D34FF48052204BD8
S3150800B73C1A8000221F4B1A700CE01F4B03EB841364
S3150800B74C9F881B4B1888FFF7B5F98742E5D001345B
S3150800B75C184B1C70174B1C78002CEED000221A7054
S3150800B76C0BE0154A02EB831292881AB9124800EBC1
S3150800B77C831007E001330F4A13700E4B1B78002B0E
S3150800B78CEFD0002088B10A4B1A88130A43EA022321
S3150800B79C8380C68015B90023036003E02B880380D9
S3150800B7AC6B88438040230372F8BD0020F8BD00BFA8
S3150800B7BC7405002076050020983D002000290CDD34
S3150800B7CC08B58AB2054B1A80054B1B68834203D011
S3150800B7DC0146184600F091FC08BD7047963D0020BE
S3150800B7EC0C370020F0B400223B4B1A703B4E1EE07F
S3150800B7FC3A4D5A001A4494002E192C5BA4B103EB4B
S3150800B80C4305AA00354D2A4452886AB10588AC42CC
S3150800B81C0AD14488A24207D10C68746089883181A0
S3150800B82C2F4A1278B27254E001332B4A13702A4B02
S3150800B83C1B78072BDCD90022274B1A700FE0274DF3
S3150800B84C5A001A4494002E192A5B2AB903EB4304AE
S3150800B85CA2002A44528832B101331F4A13701E4B78
S3150800B86C1B78072BEBD9082B28D100231D4A1370FC
S3150800B87C1D4A1370184A137013E0194A147803EB0F
S3150800B88C4305AA00154D2A44927AA61A154D2D7809
S3150800B89CAE4203DD134A1670134A137001330E4A6F
S3150800B8AC13700D4B1B78072BE7D90F4B1B780A4ADD
S3150800B8BC137003EB43039A00084E1644026833468A
S3150800B8CC43F8042B0A6872608A889A80044B1B78A2
S3150800B8DCB372F0BC704700BF7E05002080050020BF
S3150800B8ECE10500207F050020E005002010B4154B6B
S3150800B8FC1C780134E4B21C700022134B1A7019E040
S3150800B90C12485A001A4491004218415A52880A435E
S3150800B91C0DD003EB43018A000244927AA21A772AC5
S3150800B92C05DD03EB43018A000020084988500133E2
S3150800B93C054A1370044B1B78072BE1D95DF8044BA9
S3150800B94C704700BFE10500207E0500208005002019
S3150800B95C10B5324B1B88292B03D800222F4B1A8083
S3150800B96C10BD00222D4B1A802D4B9B8AB3F5807F78
S3150800B97C03D0B3F5007F3FD010BD294BDA8C294B89
S3150800B98C1B889A4249D1264B1A8D264B5B889A42BC
S3150800B99C43D1254C2146A01DFFF724FF002204F8AD
S3150800B9AC022C022204F8012C2168C4F80A10A1887A
S3150800B9BCE1811E49086820608988A18044F8100C2A
S3150800B9CC24F80C1CD4F80A1044F8161CE28924F83E
S3150800B9DC122CE288228222896282124A1188E1801C
S3150800B9EC52882281082204F80A2C062204F8092C0B
S3150800B9FC2A220A4B1A8010BD094BDA8C094B1B8874
S3150800BA0C9A420AD1064B1A8D064B5B889A4204D188
S3150800BA1C054801460630FFF7E5FE10BD083700203D
S3150800BA2C54370020503700206A370020780500204C
S3150800BA3C30B44C4BD98B8AB24FF6FF739A420CD161
S3150800BA4C484B188C4FF6FF73984206D1454B464A1D
S3150800BA5C1068186092889A8073E0444B1B88444897
S3150800BA6C00885340184209D13E4B1A8C94B23F4B6E
S3150800BA7C5B883F4840886340184206D03D4B3E4A97
S3150800BA8C1188198052885A8002E03A4B19805A80DC
S3150800BA9C00223A4B1A703A4D16E039485A001A44A5
S3150800BAAC91004518334A1488425A944209D1314AAE
S3150800BABC508803EB43018A0031490A445288904264
S3150800BACC06D001332D4A13702C4B1B78072BE4D95F
S3150800BADC082B30D1234B4FF0FF321A609A80002284
S3150800BAEC1A629A8427490868C3F806008988598116
S3150800BAFCC3F8160059831F490888D88449881985BC
S3150800BB0C1A49088898834988D9831A750121597561
S3150800BB1C9A73D973082119745A7406229A740422D2
S3150800BB2CDA74197306225A733633174A13602A22A3
S3150800BB3C164B1A8014E00B4B55F8042F1A60AA887A
S3150800BB4C9A80084B0F4A1168C3F8061092885A81D6
S3150800BB5C08221A7300225A730C4A13880E33138060
S3150800BB6C30BC70475437002050C1000850370020AD
S3150800BB7C4C370020E4050020483700207E050020BD
S3150800BB8C80050020780500201C3700200837002087
S3150800BB9C10B504464160FDF78BF9206010BD00BF57
S3150800BBAC10B50446FDF784F92368C01A63689842F1
S3150800BBBCB4BF0020012010BD352303700123437048
S3150800BBCC81700330704700BF034636220270042288
S3150800BBDC4270034A1068C3F80200981D704700BFEC
S3150800BBEC0406002037230370032343700122827056
S3150800BBFCC370062303710530704700BFFF2303701B
S3150800BC0C01307047074B828C1A80C28C5A80064BBF
S3150800BC1C028D1A80428D5A80044B028E1A80428EEF
S3150800BC2C5A807047503700204C3700204837002080
S3150800BC3C03463222027004224270034A1068C3F883
S3150800BC4C0200981D704700BF0C06002010B403466E
S3150800BC5C014400242EE01A78332A24D006D8032A65
S3150800BC6C10D0062A13D0012A21D106E0362A15D07F
S3150800BC7CFF2A21D0352A1AD10EE0D3F80200104A31
S3150800BC8C906214E0D3F802000D4A10630FE0D3F863
S3150800BC9C02000B4AD0620AE09C7808E0D3F802004E
S3150800BCAC074AD06103E0D3F80200054A10625A78B5
S3150800BCBC023213448B42CED320465DF8044B7047B0
S3150800BCCCE8050020F8B50446012303704370194BA8
S3150800BCDC9A6982700025C570174A106860602581BC
S3150800BCEC80276781154A1268E26025616561A5613E
S3150800BCFC9E693246596904F11C0000F0FEF906F1FA
S3150800BD0C18002044C6F1100229460430FCF752FCF0
S3150800BD1C4022294604F12C00FCF74CFC3A462946ED
S3150800BD2C04F16C00FCF746FC054B1868C4F8EC00EB
S3150800BD3CF8BD00BFE805002058C1000850370020A0
S3150800BD4C5CC1000838B50A4C25682846FFF7BAFFC7
S3150800BD5C012105F1F000FFF72FFFFFF743FFFFF76F
S3150800BD6C4DFF2368C11A1846FFF728FD38BD00BFDA
S3150800BD7C1C37002038B50B4C25682846FFF7A2FF60
S3150800BD8C032105F1F000FFF717FFFFF71DFFFFF77B
S3150800BD9C4FFFFFF733FF2368C11A1846FFF70EFD4E
S3150800BDAC38BD00BF1C37002010B5114B1C68237812
S3150800BDBC022B17D104220F49A01800F08FF998B955
S3150800BDCC0D4B9A69596904F11C0000F087F968B99A
S3150800BDDC2069094B5862094B198804F1F000FFF7E2
S3150800BDEC35FF10BD002010BD002010BD002010BD71
S3150800BDFC1C37002058C10008E80500200837002029
S3150800BE0C10B582B00C4C6061A1610023A3704FF68B
S3150800BE1CFF73ADF80430ADF806304FF4864101A82F
S3150800BE2CFFF778FC606010B14FF4884383800022DA
S3150800BE3C014B1A8002B010BDE8050020024B002207
S3150800BE4C1A805A80704700BF5037002038B59E4B71
S3150800BE5C1B88B3F5937F7FD010D840F20F1293420C
S3150800BE6C34D0B3F5887F01D2EBB118E1B3F5887FEE
S3150800BE7C34D040F22512934266D010E1B3F5AB7F6D
S3150800BE8C00F0BF8005D840F25512934200F0B280FC
S3150800BE9C05E1B3F5B57F00F0CE8040F26B12934204
S3150800BEAC00F0D080FBE0884B01229A704FF47A722E
S3150800BEBC1A61FFF747FF844C216904F10800FFF764
S3150800BECC67FE40F20F132380002300E00123002BAA
S3150800BEDC00F0EA804FF488727B4B1A807B4B1B78F8
S3150800BEEC13F0020F05D17A48FFF75AFE002800F026
S3150800BEFCDD80764B1B7813F0020F07D0FFF754FF43
S3150800BF0C022803D10222704B9A700CE06E4B1B6907
S3150800BF1C4EF65F22934202DC5B006B4A13616A4B56
S3150800BF2C9B78022BC5D14FF47A72674B1A61FFF7CF
S3150800BF3C21FF654C216904F10800FFF729FE40F240
S3150800BF4C25132380002300E00123002B00F0B0808A
S3150800BF5C4FF493725C4B1A805C4B1B7813F0020FF0
S3150800BF6C05D15B48FFF71CFE002800F0A380574B51
S3150800BF7C1B7813F0020F07D0FFF716FF052803D11D
S3150800BF8C0322514B9A7011E04F4B1B6942F2107207
S3150800BF9C934207DC4C4A03F57A7313619378032BA7
S3150800BFACC5D103E00020484B188038BD4648FFF73A
S3150800BFBC29FE454D288CFEF77DFD0404688CFEF79A
S3150800BFCC79FD204340084FF47A7303FB00F00028F0
S3150800BFDC01DB286103E06FF000423B4B1A613A4CD7
S3150800BFEC216904F10800FFF7D3FD40F255132380AD
S3150800BFFC002300E00123002B5ED04FF4AB72324BCA
S3150800C00C1A803348FFF7CCFD002857D02E4B022256
S3150800C01C9A704FF47A721A61FFF710FFFFF7AAFEAF
S3150800C02C294C216904F10800FFF7B2FD4FF4B573EA
S3150800C03C2380002300E00123002B41D040F26B1231
S3150800C04C214B1A80214B1B7813F0020F04D1204880
S3150800C05CFFF7A6FD002835D01C4B1B7813F0020FF2
S3150800C06C07D0FFF7A1FE052803D10322164B9A70B9
S3150800C07C11E0154B1B6942F21072934207DC124A07
S3150800C08C03F57A7313619378032BC7D103E0002069
S3150800C09C0D4B188038BD0C48FFF7B4FD89E7002214
S3150800C0AC094B1A80022038BD032038BD002038BD44
S3150800C0BC032038BD002038BD032038BD002038BD0C
S3150800C0CC032038BD002038BDE805002014370020B1
S3150800C0DCF005002008B5FFF7B9FE08BD10B5013903
S3150800C0EC0244904207D010F8013B11F8014FA342C5
S3150800C0FCF7D0181B10BD002010BD10B5431E0A44FE
S3150800C10C914204D011F8014B03F8014FF8E710BD22
S3150800C11CF8B500BFF8BC08BC9E467047F8B500BF1A
S30D0800C12CF8BC08BC9E467047EA
S3150800C1344000002000000000000000000102030483
S3150800C144060708090000000001020304FFFFFFFFB9
S3110800C154FFFF0000ADDE12236382536378
S30D0800C16028C1FF7F0100000061
S30D0800C1685D860008218200082B
S3090800C170FD81000837
S3150800C174000000002C03002094030020FC03002088
S3150800C184000000000000000000000000000000009D
S3150800C194000000000000000000000000000000008D
S3150800C1A4000000000000000000000000000000007D
S3150800C1B4000000000000000000000000000000006D
S3150800C1C4000000000000000000000000000000005D
S3150800C1D4000000000000000000000000000000004D
S3150800C1E4000000000000000000000000000000003D
S3150800C1F4000000000000000000000000000000002D
S3150800C204000000000000000000000000000000001C
S3150800C214000000000000000001000000000000000B
S3150800C2240E33CDAB34126DE6ECDE05000B000000D0
S3150800C23400000000000000000000000000000000EC
S3150800C24400000000000000000000000000000000DC
S3150800C25400000000000000000000000000000000CC
S3150800C26400000000000000000000000000000000BC
S3150800C59400000000000000000024F4001000000061
S3090800C5A40100000084
S7050800874922
